:020000040000FA
:060000000219FD0206B426
:03000B0002029658
:030013000206FDE5
:03001B0002055388
:03002B000202E3EB
:03005B0002070F8A
:030073000203186D
:1000C0000406080C10182030406080A0C09000D1B9
:1000D0007301F101FE210E211E212B213B2148211C
:1000E0005B216B217E2188219821A521BB21C8217C
:1000F000DBA6F008A67208A670088570F022A6F0AC
:1001000008A67008A67108A670088570F022E5712F
:10011000B5F002E572F608A672088570F022A6F026
:1001200008A67008A672088570F022A6F008A671CD
:1001300008A67008A670088570F022A6F008A671BF
:1001400008A671088570F022E571B5F002E572F637
:1001500008A67008A671088570F022A6F008A6709F
:1001600008A67008A671088570F022E571B5F00246
:10017000E572F608A67108A670088570F022A6F050
:1001800008A672088571F022E571B5F002E572F6F5
:1001900008A671088571F022A6F008A67008A6715D
:1001A000088571F022E571B5F002E572F608A670D7
:1001B00008A67008A670088570F022A6F008A6713F
:1001C00008A670088571F022E571B5F002E572F6B7
:1001D00008A67008A670088571F022A6F008A6701F
:1001E00008A67008A670088571F022E529A2473399
:1001F000F52875290F8075E529A24733A24633F506
:100200002875290D8066E529A24733A24633A24509
:1002100033F52875290B8054E52854F0C24C452944
:10022000C4F5287529098044E528A24813A249137A
:10023000A24A13F5287529078032E528A24813A29F
:100240004913F5287529058023E528A24813F528C8
:100250007529038017204F93204E9C204DA8204CD9
:10026000B7204BC4204AD32049DFE528C465286560
:1002700029F478D08570F023541E11CDE52823543D
:100280001E11CDE528C423541E11CDE52923541E8B
:1002900011CDA6F008220540203B0132C0D0C0E0BD
:1002A00075D01018B8CF3320850BD28585708A0899
:1002B000D0E0D0D03275A400D285C23B758E0C75CB
:1002C00089AAC2A9C289C28B758A00758C00758201
:1002D00000D2A8D2AAD0E0D0D032B285868AD0E0AF
:1002E000D0D032C0D0C0E0C2CF0541E5656009E59D
:1002F000646005756400801B756401E52360021568
:1003000023C3E554600575550080080555E5557013
:10031000021555D0E0D0D032C2AF53E67F7592FAC5
:100320007593FFC22053917FD2AF32C0D075D010E9
:10033000E52C7004E52B601EE52BA26013F528A2C6
:1003400061132528F528E52C03C2E7F52903C2E748
:100350003529F52980067528FF7529FF5155C28D6D
:10036000758A86758E097589A2D23BD2A9D2857508
:10037000A420D0D032758200752800752900752A16
:1003800000780075F000E0C0E0C395F0D0F028C31D
:10039000956978004007D24B956A4001F80582E0E4
:1003A000C0E0C395F0D0F028C3956978004007D22B
:1003B0004A956A4001F80582E0C0E0C395F0D0F0AC
:1003C00028C3956978004007D249956A4001F8052D
:1003D00082E0C0E0C395F0D0F028C3956978004072
:1003E00007D248956A4001F80582E0C0E0C395F065
:1003F000D0F028C3956978004007D247956A40013C
:10040000F80582E0C0E0C395F0D0F028C395697884
:10041000004007D246956A4001F80582E0C0E0C37B
:1004200095F0D0F028C3956978004007D245956AC9
:100430004001F80582E0C0E0C395F0D0F028C395F4
:100440006978004007D244956A4001F80582E0C00F
:10045000E0C395F0D0F028C3956978004007D243F7
:10046000956A4001F80582E0C0E0C395F0D0F0281D
:10047000C3956978004007D242956A4001F8058229
:10048000E0C0E0C395F0D0F028C39569780040073C
:10049000D241956A4001F80582E0C0E0C395F0D0F2
:1004A000F028C3956978004007D240956A4001F86A
:1004B0000582E0C0E0C395F0D0F028C395697800CC
:1004C0004007D253956A4001F80582E0C0E0C39529
:1004D000F0D0F028C3956978004007D252956A4061
:1004E00001F80582E0C0E0C395F0D0F028C395691B
:1004F00078004007D251956A4001F80582E0C0E0DB
:10050000C395F0D0F028C3956978004007D2509584
:100510006A4001F80582E528C4652865293037015D
:10052000F4652A540F22900000D2A8D2AA0522E531
:1005300022700215220522E52270021522C3E5224F
:1005400094324005755400A14C75230AD0F0D0E0D8
:10055000D0D032C2AFC2A8C28EC0D0C0E0C0F07549
:10056000D008C2CAA8CCA9CDD2CAD2AF758A00C35E
:10057000E8956CF8E9956DF9E970ABE8956E40A6E1
:10058000956F50A2E582B4109D71757099A928E508
:1005900028C39460FAE5299400FB50177B007A0089
:1005A000E96010C313500CB5520405538005F55291
:1005B000755300303702712BC2AF75E90075EA0040
:1005C000D2AF303A27C3EA94D0F8EB9407F9400B46
:1005D000E8FAE9FB203509D235A1E0303502C23511
:1005E000203902B235C3EA33FAEB33FBEB2B3B3B4A
:1005F000F9C3EB13FBEA13FAEA29FAEB3400FB30F8
:10060000E3047AFF7BFFE5255403601B202A18E5ED
:100610005C33F9EB7007C3E99A4002E9FAE53CC4A0
:10062000332AFAEB3400FBC3EA33C4540FF8EB333C
:10063000C454F048F87005EA60027801E5226002CF
:100640001522D2308854E5546003755500AC5AC366
:10065000E55A955B4002AC5BC3EC95545008EC75D1
:10066000F008A4FAABF0EB131392D5A2E7F454010F
:10067000F9EA13A2D513F4F8C3E8940FFAE9940049
:10068000FB50047A007B00C2AF88FB89FC8AE98BAF
:10069000EAD2AF1ABAFF011B885689578A588B597C
:1006A00075230A203707900000D2A8D2AAD0F0D034
:1006B000E0D0D032C0D0C0E0E58AF00582856B8BF7
:1006C000D0E0D0D032308520F00582856B8BD0E031
:1006D000D0D032F005822085FDE58AF00582856B59
:1006E0008BD0E0D0D0C28932F005823085FDE58A1A
:1006F000F00582856B8BD0E0D0D0C28932C2AA854A
:100700006B8BD28EC2CA85CC6C85CD6DD2CA32536A
:10071000E6EF327901801479038010790A800C7930
:100720001E80087964800479C880007817E4D5E0D9
:10073000FDD8FAD9F62278FF20282879A1E760238E
:10074000E548601F74FF8548F084853FF030290339
:1007500075F005A4F8C5F0600278FFC3E8955C5019
:1007600002A85C885B22C3E54794A0E5489400E5B5
:100770005B5003148001046002F55B2275E890224F
:10078000055DC3E55D9408405330EDF4A8BDA9BEF6
:10079000755D00E9FA79A0E76041EA7006E55E6000
:1007A00018800CC3E8955E600EE55E5005600A1483
:1007B00080070460FA8002E55EF55EC39568401B21
:1007C000755AC0C394044013755A80C39404400BF7
:1007D000755A40C394044003755A0022E55A241008
:1007E000500274FFF55A22743279A687F0A4C5F03E
:1007F000A2F733F55C227547007548F022C2AFC2FC
:10080000CAA8CCA9CDAA4130CF010AD2CAD2AFC35F
:10081000EA13FAE913F9E813F8AB42AC43884289CA
:1008200043C3E89BF8E99C20280A547FF9302C0246
:10083000211B8040AD448A44F9EA9D547FFA60064A
:1008400078FF79FF8013AE45AF468B458C46A842B2
:10085000A943C3E89EF8E99FF9C3E54813FBE547C0
:1008600013FAE82AF547E93BF54850087547FF7544
:1008700048FF804DAA47AB48AC47AD487E047F0295
:10088000C3EB9404400D1E1FC3EB940840052029C0
:10089000021E1FC3ED13FDEC13FCDEF7C3EA9CFA46
:1008A000EB9DFBEF6009C3E913F9E813F8DFF7EA02
:1008B00028FAEB39FB8A478B4850067BFF8B478B26
:1008C00048C3EB94025002D22C3028047F03801CD2
:1008D0007892E6FFC3E53D948240110FC3E53D9455
:1008E000A040010FC3EF940640027F057E02E54859
:1008F000C4540FF9E548C454F0F8E547C4540F2830
:10090000F8C3E89EFAE99400FB4009C3EA9401EBBE
:10091000940050047A01E4FB020967AA47AB48EB54
:10092000C4FEEAC4540F4EFCC3EA9CFAEB9400FBED
:10093000C3E813C313F8EA28FAEB3400FB8A478BA9
:1009400048C3EB94024002C22C7802EBC4FE7B0049
:10095000EAC4540F4EFAC3EA98FA4005C394015012
:10096000027A017892E6FFC2AF85472B85482CD2E8
:10097000AF3020022167854E92854F93D22043E607
:1009800080C3E49AF8E49BF9C3E833F8E933F9301B
:100990002C03020A06E8FAE9FBD3E913FDE813FC8D
:1009A000884E894FC3EF94036038EF20E00CE82CA9
:1009B000F8E93DF9ECFAEDFB8013E828F8E939F99C
:1009C000C3E82401F8E93400F97AFF7BFFC3EF9410
:1009D00003400F8A508B51884A894B8C4C8D4D02B5
:1009E0000A3B885089518A4A8B4B8C4C8D4D30285C
:1009F000127550F07551FF754CF0754DFF754EF046
:100A0000754FFF020A3BE8FAD3E813FC884EC3EFA8
:100A100094036021EF20E007E82CF8ECFA4126E887
:100A2000282401F87AFFC3EF940340098A50884ACA
:100A30008C4C020A3B88508A4A8C4C302002413B45
:100A4000753A02D22043E680E5255403602DA8477D
:100A5000A948C3E913F9E813F8302804E92440F958
:100A6000C2AF53E67F759100C3E498F594E499F51D
:100A700095759104D22043E680D2AF22D2217549E8
:100A800000752000302B03752040419AD221754912
:100A900000752040302B0375200078017901202C4F
:100AA00020E52554036002C2217914E548C3137080
:100AB0000104F8C3941440027814302804781B7998
:100AC0001BC3E833F8C3E933F9202010E549600C73
:100AD000302803D53A04D222614D51430549E59BA4
:100AE0005440B52002613730280908C3E899400115
:100AF0001841C920210A08C3E8994002419A41C916
:100B0000C22153E67F759100302C117594007595C4
:100B1000F0759104D22043E680020A9AE5487EFFF0
:100B2000C3334009C3334005C3334001FEC3E49ED1
:100B3000759400F5956111C3E53994015002419A0D
:100B4000302102419AD802614B41C9C222C2AF533F
:100B5000E67F759100855094855195759104854A7D
:100B600092854B93D22043E680D2AFE525540360B3
:100B7000072029020539801030220D202B0A202160
:100B800007158115810215CA2278003021027801EB
:100B9000E53D75F007A4F9E5F028F5F0E9A2F013BA
:100BA000A2F113A2F213F53DC394785003753D787A
:100BB000C3E53D953E4009C290C292C29475D53FAF
:100BC00030200261C0854C92854D93D22043E6804F
:100BD00022203811C2AFC293C29575D50FD291D2DF
:100BE000AF759F0322C2AFC291C29375D53CD29517
:100BF000D2AF759F032220381DC2AFC293C2957534
:100C0000D8008558F98559FA75D53375D840D291F1
:100C1000D2AF759F1322C2AFC291C29375D800851F
:100C200058F98559FA75D53375D840D295D2AF7534
:100C30009F2322203811C2AFC291C29375D533D2FF
:100C400095D2AF759F2322C2AFC293C29575D5339B
:100C5000D291D2AF759F132220381DC2AFC291C26C
:100C60009375D8008558F98559FA75D53C75D840E3
:100C7000D295D2AF759F0322C2AFC293C29575D8E9
:100C8000008558F98559FA75D50F75D840D291D29B
:100C9000AF759F0322203811C2AFC291C29575D59E
:100CA0003CD293D2AF759F1322C2AFC291C2957549
:100CB000D50FD293D2AF759F232220381DC2AFC269
:100CC00091C29575D8008558F98559FA75D50F7573
:100CD000D840D293D2AF759F2322C2AFC291C295A2
:100CE00075D8008558F98559FA75D53C75D840D224
:100CF00093D2AF759F13227A147B7880127A107B7F
:100D00008C800C7A0D7BB480067A0B7BC88000E562
:100D100063D5E001227902E4C293D5E0FDD292D5F9
:100D2000E0FDC292D5E0FDD293D5E0FDE920E002DE
:100D3000D29030E002D294E563D5E0FDE920E002F4
:100D4000C29030E002C2947496D5E0FDD9C9EAF8A9
:100D5000D5E0FDD8FBDBB8C29322C290C292C29408
:100D6000C291C293C29575D53F22788076FF0876EE
:100D7000FF0876FF0876FF0876FF0876FF087609F9
:100D80000876FF087601788C76010876FF0876FFF2
:100D90000876FF0876FF0876FF0876030876FF08D6
:100DA00076FF0876FF0876250876D008762808763C
:100DB000500876040876FF0876020876FF08767AEF
:100DC0000876FF0876070876010876FF0876FF08A0
:100DD000760008760022FA75F00CA4ABF0EAC33373
:100DE000F8740133F9E8C333F8E933F9E8C32BF8B1
:100DF000E93400F9E8C333F8E933F9227888E6C327
:100E00009403D23A5002C23AC238E630E102D238F4
:100E1000A23892397886E6149000C09378A6F678C6
:100E200086E6F53FC394025003753F02789CE67551
:100E30003EFFB40203753EA0B40303753E8278A062
:100E4000E6F8600674282409D8FCF5687896E6B1BF
:100E5000D688318932789EE6B1D68833893478973E
:100E6000E6B1D688358936B15A223036117A007B00
:100E7000007CFF7D007E00D1D08B608A5F22303AFB
:100E8000227896E6FA7B00789EE6FC7D00C3EA3382
:100E9000FAEB33FBC3EC33FCED33FD7E0AD1D08B90
:100EA000628A617896303A02789EE6FA7B007897FB
:100EB000E6FC7D007E00303A10C3EA33FAEB33FBE8
:100EC000C3EC33FCED33FD7E0AD1D08B608A5F2208
:100ED000C3EC9EFCED9400FDC3EC9AFCED9BFDC3BE
:100EE000EC9423ED940050047C237D00C3EC94FF2C
:100EF000ED940140047CFF7D017BFF0B7A000AEA40
:100F00007009C3EC33FCED33FD80F0EC8AF0A4AE45
:100F1000F0ED8AF0A42E947C40E4EAF460DD22D265
:100F200036D16A12071F12071F7A007B007C10124D
:100F30000717E5542AFA74003BFBDCF37C04C3EB8F
:100F400013FBEA13FADCF7FFEB60027FFFC236D136
:100F50006A2278A5E6F954037000E9540C7000E9A0
:100F600054307000E954C0700022758851758E0CA1
:100F70007589AA758C00758D00758E0C756B3C7526
:100F80006920756A1E303703756A1B756E4E756F62
:100F9000437570FF7571EC7572DD22758851758E21
:100FA0000C7589AA758C00758D00758E0C756B009B
:100FB000756940756A3C303703756A36756E9D7584
:100FC0006F877570EC7571CB7572AB22741E2085BE
:100FD00015C0D0C0E0740AD5E0FDD0E0D0D02085A7
:100FE000EBD5E0EDC322C0D0C0E0740AD5E0FDD05F
:100FF000E0D0D03085D6D5E0EDD322756600756798
:10100000007597DE7597AD7581AF43FF8075EF066C
:1010100075A900120D5A7580FF75F1F075A4007561
:1010200080FF75D4FF75900075F23F75A53F7590F0
:101030000075D53F75A60175E34075E202120D5AA1
:10104000E4F8F6D8FD120D6AB1FE78988663753023
:1010500001C2AF120727120CF712071F120CFD1264
:10106000071F120D0312071F120F52C2AF75660041
:1010700075670078FA79FA308516D9FBD8F775A923
:101080001375A71075C10075A700756500021C00D7
:10109000120DFC120E6A78988663120D5A75A7100D
:1010A00075C13075A70075A90375650175C804750C
:1010B000910475D84075D90875F781759E037596AA
:1010C0000275DA4275DB4275A82375E68075B803B0
:1010D000759B80759D0075D10C75BCB975BB10757D
:1010E000E88075B201120713753C00C23012072761
:1010F000C231C232C233C234755200755300D23489
:10110000120FCC9237C23B752B00752C0075E4D5BD
:1011100030370375E45D120F6AC2A9D2ABD2AAD2EE
:10112000AF752232120723755200755300C3E522B2
:1011300094024018120F9B75223212072375520039
:10114000755300C3E52294024002016B1207172079
:101150003002016BE5546002016BC2AF120CF71252
:101160000CF7120CF7D2AF120727203403303A03E2
:10117000021219120717788CE6C394015002411924
:10118000E530C39401500241197566A57567F17F7A
:1011900002D236120E6A120723C2AFC236120E6A8C
:1011A000C3E554947FD2AF4070120713C2AF120D43
:1011B00009D2AFDFDC120F1FC3EF7897F6120727B3
:1011C000D1EB7F0AD236120E6A120723C2AFC236A3
:1011D000120E6AC3E554947FD2AF50E6120713C2D1
:1011E000AF120CF712071B120CF7D2AFDFD6120F9B
:1011F0001FEF24037896F6F87997E7C3942340030A
:10120000985006E824237897F6120727D145F11A5B
:10121000120723120E6A02106B75660075670012C2
:101220000723E5546002016BC2AF120D09120D09CC
:10123000120D09D2AF120727753000752B00752CDF
:1012400000E4F537F5380537E537F4703F053878B1
:101250009AE67819146012783214600D787D146063
:101260000878FA146003753800C3E53898401D12F9
:101270000D5A120713153875370078998663C2AF77
:10128000120D09D2AF7898866312072312071BE567
:10129000237002016BC3E5549401500AC3E55294D4
:1012A000015016021246120723E523700302106B49
:1012B00075520075530002145BC3E5529401701718
:1012C000C2AF120D5A78998663120CF7789886632C
:1012D000D2AF120723814DC3E55294027017C2AFFB
:1012E000120D5A78998663120CFD78988663D2AFF6
:1012F000120723814DC3E55294037017C2AF120D3C
:101300005A78998663120D0378988663D2AF1207D4
:1013100023814DC3E55294047017C2AF120D5A7861
:10132000998663120D0978988663D2AF12072381DC
:101330004DC3E55294057017C2AF120D5A789986C5
:1013400063120D0978988663D2AF120723814DC3CB
:10135000E55294077019C3E5539406500241957401
:1013600001303A0274037888F6C238C239814DC31D
:10137000E55294087019C3E55394065002419574E0
:1013800002303A0274047888F6D238D239814DC3DB
:10139000E55294097017C3E5539406500241953005
:1013A0003A0BC37888E69402F6C23A814DC3E552FF
:1013B000940A7016C3E553940650024195203A0AE8
:1013C0007888E62402F6D23A814DC3E5529414702F
:1013D00025C3E553940650024195C2AF901A0B7491
:1013E0000093D2AF7888F613C238C2394002D2389F
:1013F0004002D2398057C3E55294157038C3E55383
:101400009406404FC2AF901A0B740093D2AFF8B855
:1014100001027402B802027401B803027404B80431
:101420000274037888F613C238C2394002D23840B9
:1014300002D2398018C3E552940C70117566A575F7
:1014400067F1C3E5539406400AD145D2AF75520007
:101450007553007566007567004195C2AF120D5A4D
:10146000E4D2AFE4F55DF524F525F53D755D081290
:10147000071312077C30EDFDA8BDA9BEE97001F885
:10148000885E120780755D08C2AF1207E7855C5A57
:10149000855C5BD2AF75A71075C13075A70075A9C3
:1014A00003756501303A07C238303502D238D22888
:1014B000753900120C95120CBA1207F61207FD12BC
:1014C00007F61207FD1207F6120A8C120B89120B8F
:1014D000D11207FD120A7C202C03120736302C0390
:1014E000120766120B89120BF61207FD120A8C12F4
:1014F0000B89120C331207FD120A7C120B89120C95
:10150000581207FD120A8C120B89120C951207FD56
:1015100012077C120A7C120B89120CBA1207801275
:1015200007FD302827855C5A79187A0CC3E539996C
:10153000400EC228D2298A3B855C5A855C5B800CB0
:10154000C3E554940140030214C8A1D230291F20DE
:101550002B1CE53B147006C229D22A81C8F53B201A
:101560003A07C3E554940140030214C88064753CF3
:1015700000203A0F78FA79A4E760027803C3E555B2
:1015800098504FE523604B303A1720380520350737
:10159000800F303502800A202B07D22B855C5A81C0
:1015A000F878F0302B05855C5A7820C3E5489850D0
:1015B000030214C8302B1BC22BC238303502D2387C
:1015C000D229753B12855C5A81C8053CE5546002FE
:1015D000A1D5753C00C2AF120D5A752500D2AF12CD
:1015E0000723120D5A75240078A4E66006D291D222
:1015F00093D295C3E53C94044002016B413B901AA1
:101600000D7820D17EE520B4550AA3D17EE520B423
:10161000AA0280137566A57567F1120D6AD145752A
:101620006600756700801D901A0378807B0AD17E62
:10163000A308DBFA901A0F788C7B1AD17EA308DB03
:10164000FA901A2922C2AFD1C1D19E901A0074100B
:10165000D183A3744DD183A37421D183901A0378CD
:10166000807B0AD182A308DBFA901A0F788C7B1A50
:10167000D182A308DBFAD1D4D1B2901A2922E49303
:10168000F622E6438F01538FFDFFC3E583941C4090
:101690000122EF8566B78567B7F0538FFE22438F2F
:1016A00002438F018566B78567B7901A0DF0538F97
:1016B000FC22901A0D7455D183901A0E74AAD1830E
:1016C000227A3079D07820901A40D17EE520F7092F
:1016D000A3DAF7227A3079D0901A40E7D18309A3B0
:1016E000DAF9227C05120727DCFB22C2AF120CF7C5
:1016F000120CFD120D03120D0912071B120CF7122A
:101700000CFD120D03120D0912071B120CF7120C1F
:10171000FD120D03120D09D2AF22C2AF120D091234
:101720000D03120CFD120CF712071B120D09120DFE
:1017300003120CFD120CF712071B120D09120D03F8
:09174000120CFD120CF7D2AF22CD
:1019FD00020FFB104D21FFFFFFFFFFFF09FF01FF4E
:101A0D0055AA01FFFFFFFFFF03FFFFFF25D0285061
:0D1A1D0004FF02FF7AFF0701FFFF0000FF3A
:101A400023475F485F31352320202020202020209D
:101A500023424C48454C492445464D3842323123B7
:101A60002020202020202020202020202020202076
:101C0000C2AFC2D37597DE7597AD7581C075A90057
:101C100043FF80752438752503B1EA7529A5752A17
:101C2000F143F12053A4DFD28575D4FF75E3407DE5
:101C3000FA780379E67C10752200752300901DF771
:101C40007B06752498752501E4308510C0E0E430EA
:101C5000850AD5E0FAD0E0D5E0EF806D208508D880
:101C6000FBD9F9DCF781C9308508D8FBD9F9DCF755
:101C700081C9B1AAE493A3C39A6004DDB481C9DB2E
:101C8000DBB19C600281317B08E493FAA3B17DDB78
:101C9000F87A30B17D752200752300B19CEAFCEB27
:101CA000FDC3ED94FE400EB19C8A278B28ED30E0F9
:101CB000048A828B83B19C7AC270D8C3ED94FE6093
:101CC0001950CEBD0029EC600F7520007521FF75FD
:101CD0002900752A000200008100A827A928080908
:101CE000D804D90281ECB1A0EAF281E00D81B5C33C
:101CF000ED94035051EDA2E092007AC5C3E58294C1
:101D000000E583941C508C200010438F02438F0108
:101D10008529B7852AB7F0300027A827A928080900
:101D2000438F01538FFDD804D902A141C3E58394A9
:101D30001C4003A3A126E28529B7852AB7F0A3A1F9
:101D400026538FFC81917AC1BD030CE493A3FAB1B1
:101D500061DCF8B15981918193AA22AB23B17DEB6B
:101D6000FAEA6222752608C3E52313F523E5221358
:101D7000F52250066323A0632201D526EAB1EAB119
:101D8000EA75260AEAF4200102D285300102C285F2
:101D9000B1EAC3134002C201D526EB22B1A0EAFB8F
:101DA000208502A1A0308502A1A5752608AE24AF2A
:101DB00025C3EF13FFEE13FEB1EEB1EAC3EA133011
:101DC00085024480FA30E703632201C3E52313F55B
:101DD00023E52213F52250066323A0632201D526B2
:101DE000D9E52265236523F52222AE24AF250E0F07
:101DF000DEFEDFFCD20122424C48656C693437318B
:051E000064E8B20601D8
:00000001FF
